Archive member included because of file (symbol)

c:/winavr-20080610/bin/../lib/gcc/avr/4.3.0/avr35\libgcc.a(_mulhi3.o)
                              USB10.o (__mulhi3)
c:/winavr-20080610/bin/../lib/gcc/avr/4.3.0/avr35\libgcc.a(_udivmodhi4.o)
                              USB10.o (__udivmodhi4)
c:/winavr-20080610/bin/../lib/gcc/avr/4.3.0/avr35\libgcc.a(_udivmodsi4.o)
                              USB10.o (__udivmodsi4)
c:/winavr-20080610/bin/../lib/gcc/avr/4.3.0/avr35\libgcc.a(_exit.o)
                              c:/winavr-20080610/bin/../lib/gcc/avr/4.3.0/../../../../avr/lib/avr35/crtusb162.o (exit)
c:/winavr-20080610/bin/../lib/gcc/avr/4.3.0/avr35\libgcc.a(_copy_data.o)
                              USB10.o (__do_copy_data)
c:/winavr-20080610/bin/../lib/gcc/avr/4.3.0/avr35\libgcc.a(_clear_bss.o)
                              USB10.o (__do_clear_bss)

Allocating common symbols
Common symbol       size              file

outputBuffer        0x14              USB10.o
USB_IsInitialized   0x1               ../../MyUSB/Drivers/USB/HighLevel/USBTask.o
USB_CurrentlySelfPowered
                    0x1               ../../MyUSB/Drivers/USB/LowLevel/DevChapter9.o
inputBuffer         0x14              USB10.o
USB_RemoteWakeupEnabled
                    0x1               ../../MyUSB/Drivers/USB/LowLevel/DevChapter9.o
Tx_Buffer           0x85              USB10.o
USB_IsConnected     0x1               ../../MyUSB/Drivers/USB/HighLevel/USBTask.o
Scheduler_TotalTasks
                    0x1               ../../MyUSB/Scheduler/Scheduler.o
Rx_Buffer           0x85              USB10.o
USB_ConfigurationNumber
                    0x1               ../../MyUSB/Drivers/USB/LowLevel/DevChapter9.o
Scheduler_TickCounter
                    0x2               ../../MyUSB/Scheduler/Scheduler.o

Discarded input sections

 .data          0x00000000        0x0 c:/winavr-20080610/bin/../lib/gcc/avr/4.3.0/../../../../avr/lib/avr35/crtusb162.o
 .bss           0x00000000        0x0 c:/winavr-20080610/bin/../lib/gcc/avr/4.3.0/../../../../avr/lib/avr35/crtusb162.o
 .text          0x00000000        0x0 USB10.o
 .text.testReset
                0x00000000        0x0 USB10.o
 .text.uart_puts
                0x00000000        0x0 USB10.o
 .text.Print_Int
                0x00000000        0x0 USB10.o
 .progmem.data  0x00000000        0x0 USB10.o
 .text          0x00000000        0x0 Descriptors.o
 .data          0x00000000        0x0 Descriptors.o
 .bss           0x00000000        0x0 Descriptors.o
 .text          0x00000000        0x0 RingBuff.o
 .data          0x00000000        0x0 RingBuff.o
 .bss           0x00000000        0x0 RingBuff.o
 .text          0x00000000        0x0 I2C_bitbanged.o
 .data          0x00000000        0x0 I2C_bitbanged.o
 .bss           0x00000000        0x0 I2C_bitbanged.o
 .text.I2C_RepeatedStart
                0x00000000        0x0 I2C_bitbanged.o
 .text.Delay    0x00000000        0x0 I2C_bitbanged.o
 .text          0x00000000        0x0 StepDirLineCoding.o
 .data          0x00000000        0x0 StepDirLineCoding.o
 .bss           0x00000000        0x0 StepDirLineCoding.o
 .text          0x00000000        0x0 ../../MyUSB/Scheduler/Scheduler.o
 .data          0x00000000        0x0 ../../MyUSB/Scheduler/Scheduler.o
 .bss           0x00000000        0x0 ../../MyUSB/Scheduler/Scheduler.o
 .text.Scheduler_HasDelayElapsed
                0x00000000        0x0 ../../MyUSB/Scheduler/Scheduler.o
 .text.Scheduler_SetGroupTaskMode
                0x00000000        0x0 ../../MyUSB/Scheduler/Scheduler.o
 .text          0x00000000        0x0 ../../MyUSB/Drivers/AT90USBXXX/Serial.o
 .data          0x00000000        0x0 ../../MyUSB/Drivers/AT90USBXXX/Serial.o
 .bss           0x00000000        0x0 ../../MyUSB/Drivers/AT90USBXXX/Serial.o
 .text.Serial_Init
                0x00000000        0x0 ../../MyUSB/Drivers/AT90USBXXX/Serial.o
 .text.Serial_TxString_P
                0x00000000        0x0 ../../MyUSB/Drivers/AT90USBXXX/Serial.o
 .text.Serial_TxString
                0x00000000        0x0 ../../MyUSB/Drivers/AT90USBXXX/Serial.o
 .text          0x00000000        0x0 ../../MyUSB/Drivers/USB/LowLevel/LowLevel.o
 .data          0x00000000        0x0 ../../MyUSB/Drivers/USB/LowLevel/LowLevel.o
 .bss           0x00000000        0x0 ../../MyUSB/Drivers/USB/LowLevel/LowLevel.o
 .text          0x00000000        0x0 ../../MyUSB/Drivers/USB/LowLevel/Endpoint.o
 .bss           0x00000000        0x0 ../../MyUSB/Drivers/USB/LowLevel/Endpoint.o
 .text.Endpoint_ClearEndpoints
                0x00000000        0x0 ../../MyUSB/Drivers/USB/LowLevel/Endpoint.o
 .text.Endpoint_WaitUntilReady
                0x00000000        0x0 ../../MyUSB/Drivers/USB/LowLevel/Endpoint.o
 .text.Endpoint_Discard_Stream
                0x00000000        0x0 ../../MyUSB/Drivers/USB/LowLevel/Endpoint.o
 .text.Endpoint_Write_Stream_LE
                0x00000000        0x0 ../../MyUSB/Drivers/USB/LowLevel/Endpoint.o
 .text.Endpoint_Write_Stream_BE
                0x00000000        0x0 ../../MyUSB/Drivers/USB/LowLevel/Endpoint.o
 .text.Endpoint_Read_Stream_LE
                0x00000000        0x0 ../../MyUSB/Drivers/USB/LowLevel/Endpoint.o
 .text.Endpoint_Read_Stream_BE
                0x00000000        0x0 ../../MyUSB/Drivers/USB/LowLevel/Endpoint.o
 .text.Endpoint_Write_Control_Stream_BE
                0x00000000        0x0 ../../MyUSB/Drivers/USB/LowLevel/Endpoint.o
 .text.Endpoint_Read_Control_Stream_BE
                0x00000000        0x0 ../../MyUSB/Drivers/USB/LowLevel/Endpoint.o
 .text          0x00000000        0x0 ../../MyUSB/Drivers/USB/LowLevel/DevChapter9.o
 .data          0x00000000        0x0 ../../MyUSB/Drivers/USB/LowLevel/DevChapter9.o
 .bss           0x00000000        0x0 ../../MyUSB/Drivers/USB/LowLevel/DevChapter9.o
 .text          0x00000000        0x0 ../../MyUSB/Drivers/USB/HighLevel/USBTask.o
 .data          0x00000000        0x0 ../../MyUSB/Drivers/USB/HighLevel/USBTask.o
 .bss           0x00000000        0x0 ../../MyUSB/Drivers/USB/HighLevel/USBTask.o
 .text          0x00000000        0x0 ../../MyUSB/Drivers/USB/HighLevel/USBInterrupt.o
 .data          0x00000000        0x0 ../../MyUSB/Drivers/USB/HighLevel/USBInterrupt.o
 .bss           0x00000000        0x0 ../../MyUSB/Drivers/USB/HighLevel/USBInterrupt.o
 .text          0x00000000        0x0 ../../MyUSB/Drivers/USB/HighLevel/Events.o
 .data          0x00000000        0x0 ../../MyUSB/Drivers/USB/HighLevel/Events.o
 .bss           0x00000000        0x0 ../../MyUSB/Drivers/USB/HighLevel/Events.o
 .text          0x00000000        0x0 ../../MyUSB/Drivers/USB/HighLevel/StdDescriptors.o
 .data          0x00000000        0x0 ../../MyUSB/Drivers/USB/HighLevel/StdDescriptors.o
 .bss           0x00000000        0x0 ../../MyUSB/Drivers/USB/HighLevel/StdDescriptors.o
 .text.USB_GetDescriptor
                0x00000000        0x0 ../../MyUSB/Drivers/USB/HighLevel/StdDescriptors.o
 .text          0x00000000        0x0 c:/winavr-20080610/bin/../lib/gcc/avr/4.3.0/avr35\libgcc.a(_mulhi3.o)
 .data          0x00000000        0x0 c:/winavr-20080610/bin/../lib/gcc/avr/4.3.0/avr35\libgcc.a(_mulhi3.o)
 .bss           0x00000000        0x0 c:/winavr-20080610/bin/../lib/gcc/avr/4.3.0/avr35\libgcc.a(_mulhi3.o)
 .text          0x00000000        0x0 c:/winavr-20080610/bin/../lib/gcc/avr/4.3.0/avr35\libgcc.a(_udivmodhi4.o)
 .data          0x00000000        0x0 c:/winavr-20080610/bin/../lib/gcc/avr/4.3.0/avr35\libgcc.a(_udivmodhi4.o)
 .bss           0x00000000        0x0 c:/winavr-20080610/bin/../lib/gcc/avr/4.3.0/avr35\libgcc.a(_udivmodhi4.o)
 .text          0x00000000        0x0 c:/winavr-20080610/bin/../lib/gcc/avr/4.3.0/avr35\libgcc.a(_udivmodsi4.o)
 .data          0x00000000        0x0 c:/winavr-20080610/bin/../lib/gcc/avr/4.3.0/avr35\libgcc.a(_udivmodsi4.o)
 .bss           0x00000000        0x0 c:/winavr-20080610/bin/../lib/gcc/avr/4.3.0/avr35\libgcc.a(_udivmodsi4.o)
 .text          0x00000000        0x0 c:/winavr-20080610/bin/../lib/gcc/avr/4.3.0/avr35\libgcc.a(_exit.o)
 .data          0x00000000        0x0 c:/winavr-20080610/bin/../lib/gcc/avr/4.3.0/avr35\libgcc.a(_exit.o)
 .bss           0x00000000        0x0 c:/winavr-20080610/bin/../lib/gcc/avr/4.3.0/avr35\libgcc.a(_exit.o)
 .text.libgcc   0x00000000        0x0 c:/winavr-20080610/bin/../lib/gcc/avr/4.3.0/avr35\libgcc.a(_exit.o)
 .text          0x00000000        0x0 c:/winavr-20080610/bin/../lib/gcc/avr/4.3.0/avr35\libgcc.a(_copy_data.o)
 .data          0x00000000        0x0 c:/winavr-20080610/bin/../lib/gcc/avr/4.3.0/avr35\libgcc.a(_copy_data.o)
 .bss           0x00000000        0x0 c:/winavr-20080610/bin/../lib/gcc/avr/4.3.0/avr35\libgcc.a(_copy_data.o)
 .text.libgcc   0x00000000        0x0 c:/winavr-20080610/bin/../lib/gcc/avr/4.3.0/avr35\libgcc.a(_copy_data.o)
 .text          0x00000000        0x0 c:/winavr-20080610/bin/../lib/gcc/avr/4.3.0/avr35\libgcc.a(_clear_bss.o)
 .data          0x00000000        0x0 c:/winavr-20080610/bin/../lib/gcc/avr/4.3.0/avr35\libgcc.a(_clear_bss.o)
 .bss           0x00000000        0x0 c:/winavr-20080610/bin/../lib/gcc/avr/4.3.0/avr35\libgcc.a(_clear_bss.o)
 .text.libgcc   0x00000000        0x0 c:/winavr-20080610/bin/../lib/gcc/avr/4.3.0/avr35\libgcc.a(_clear_bss.o)

Memory Configuration

Name             Origin             Length             Attributes
text             0x00000000         0x00020000         xr
data             0x00800060         0x0000ffa0         rw !x
eeprom           0x00810000         0x00010000         rw !x
fuse             0x00820000         0x00000400         rw !x
lock             0x00830000         0x00000400         rw !x
signature        0x00840000         0x00000400         rw !x
*default*        0x00000000         0xffffffff

Linker script and memory map

Address of section .data set to 0x800100
LOAD c:/winavr-20080610/bin/../lib/gcc/avr/4.3.0/../../../../avr/lib/avr35/crtusb162.o
LOAD USB10.o
LOAD Descriptors.o
LOAD RingBuff.o
LOAD I2C_bitbanged.o
LOAD StepDirLineCoding.o
LOAD ../../MyUSB/Scheduler/Scheduler.o
LOAD ../../MyUSB/Drivers/AT90USBXXX/Serial.o
LOAD ../../MyUSB/Drivers/USB/LowLevel/LowLevel.o
LOAD ../../MyUSB/Drivers/USB/LowLevel/Endpoint.o
LOAD ../../MyUSB/Drivers/USB/LowLevel/DevChapter9.o
LOAD ../../MyUSB/Drivers/USB/HighLevel/USBTask.o
LOAD ../../MyUSB/Drivers/USB/HighLevel/USBInterrupt.o
LOAD ../../MyUSB/Drivers/USB/HighLevel/Events.o
LOAD ../../MyUSB/Drivers/USB/HighLevel/StdDescriptors.o
LOAD c:/winavr-20080610/bin/../lib/gcc/avr/4.3.0/../../../../avr/lib/avr35\libm.a
LOAD c:/winavr-20080610/bin/../lib/gcc/avr/4.3.0/avr35\libgcc.a
LOAD c:/winavr-20080610/bin/../lib/gcc/avr/4.3.0/../../../../avr/lib/avr35\libc.a
LOAD c:/winavr-20080610/bin/../lib/gcc/avr/4.3.0/avr35\libgcc.a

.hash
 *(.hash)

.dynsym
 *(.dynsym)

.dynstr
 *(.dynstr)

.gnu.version
 *(.gnu.version)

.gnu.version_d
 *(.gnu.version_d)

.gnu.version_r
 *(.gnu.version_r)

.rel.init
 *(.rel.init)

.rela.init
 *(.rela.init)

.rel.text
 *(.rel.text)
 *(.rel.text.*)
 *(.rel.gnu.linkonce.t*)

.rela.text
 *(.rela.text)
 *(.rela.text.*)
 *(.rela.gnu.linkonce.t*)

.rel.fini
 *(.rel.fini)

.rela.fini
 *(.rela.fini)

.rel.rodata
 *(.rel.rodata)
 *(.rel.rodata.*)
 *(.rel.gnu.linkonce.r*)

.rela.rodata
 *(.rela.rodata)
 *(.rela.rodata.*)
 *(.rela.gnu.linkonce.r*)

.rel.data
 *(.rel.data)
 *(.rel.data.*)
 *(.rel.gnu.linkonce.d*)

.rela.data
 *(.rela.data)
 *(.rela.data.*)
 *(.rela.gnu.linkonce.d*)

.rel.ctors
 *(.rel.ctors)

.rela.ctors
 *(.rela.ctors)

.rel.dtors
 *(.rel.dtors)

.rela.dtors
 *(.rela.dtors)

.rel.got
 *(.rel.got)

.rela.got
 *(.rela.got)

.rel.bss
 *(.rel.bss)

.rela.bss
 *(.rela.bss)

.rel.plt
 *(.rel.plt)

.rela.plt
 *(.rela.plt)

.text           0x00000000     0x1830
 *(.vectors)
 .vectors       0x00000000       0x74 c:/winavr-20080610/bin/../lib/gcc/avr/4.3.0/../../../../avr/lib/avr35/crtusb162.o
                0x00000000                __vectors
                0x00000000                __vector_default
 *(.vectors)
 *(.progmem.gcc*)
 *(.progmem*)
 .progmem.data  0x00000074       0x9f Descriptors.o
                0x000000cd                ManufacturerString
                0x000000c9                LanguageString
                0x00000074                DeviceDescriptor
                0x000000e7                ProductString
                0x00000086                ConfigurationDescriptor
                0x00000114                . = ALIGN (0x2)
 *fill*         0x00000113        0x1 00
                0x00000114                __trampolines_start = .
 *(.trampolines)
 .trampolines   0x00000114        0x0 linker stubs
 *(.trampolines*)
                0x00000114                __trampolines_end = .
 *(.jumptables)
 *(.jumptables*)
 *(.lowtext)
 *(.lowtext*)
                0x00000114                __ctors_start = .
 *(.ctors)
                0x00000114                __ctors_end = .
                0x00000114                __dtors_start = .
 *(.dtors)
                0x00000114                __dtors_end = .
 SORT(*)(.ctors)
 SORT(*)(.dtors)
 *(.init0)
 .init0         0x00000114        0x0 c:/winavr-20080610/bin/../lib/gcc/avr/4.3.0/../../../../avr/lib/avr35/crtusb162.o
                0x00000114                __init
 *(.init0)
 *(.init1)
 *(.init1)
 *(.init2)
 .init2         0x00000114        0xc c:/winavr-20080610/bin/../lib/gcc/avr/4.3.0/../../../../avr/lib/avr35/crtusb162.o
 *(.init2)
 *(.init3)
 *(.init3)
 *(.init4)
 .init4         0x00000120       0x16 c:/winavr-20080610/bin/../lib/gcc/avr/4.3.0/avr35\libgcc.a(_copy_data.o)
                0x00000120                __do_copy_data
 .init4         0x00000136       0x10 c:/winavr-20080610/bin/../lib/gcc/avr/4.3.0/avr35\libgcc.a(_clear_bss.o)
                0x00000136                __do_clear_bss
 *(.init4)
 *(.init5)
 *(.init5)
 *(.init6)
 *(.init6)
 *(.init7)
 *(.init7)
 *(.init8)
 *(.init8)
 *(.init9)
 .init9         0x00000146        0x6 c:/winavr-20080610/bin/../lib/gcc/avr/4.3.0/../../../../avr/lib/avr35/crtusb162.o
 *(.init9)
 *(.text)
 .text          0x0000014c        0x2 c:/winavr-20080610/bin/../lib/gcc/avr/4.3.0/../../../../avr/lib/avr35/crtusb162.o
                0x0000014c                __vector_22
                0x0000014c                __vector_28
                0x0000014c                __vector_1
                0x0000014c                __vector_24
                0x0000014c                __vector_12
                0x0000014c                __bad_interrupt
                0x0000014c                __vector_6
                0x0000014c                __vector_3
                0x0000014c                __vector_13
                0x0000014c                __vector_17
                0x0000014c                __vector_19
                0x0000014c                __vector_7
                0x0000014c                __vector_27
                0x0000014c                __vector_5
                0x0000014c                __vector_4
                0x0000014c                __vector_9
                0x0000014c                __vector_2
                0x0000014c                __vector_21
                0x0000014c                __vector_15
                0x0000014c                __vector_8
                0x0000014c                __vector_26
                0x0000014c                __vector_14
                0x0000014c                __vector_10
                0x0000014c                __vector_16
                0x0000014c                __vector_18
                0x0000014c                __vector_20
                0x0000014e                . = ALIGN (0x2)
 *(.text.*)
 .text.ReconfigureUSART
                0x0000014e       0x70 USB10.o
                0x0000014e                ReconfigureUSART
 .text.__vector_25
                0x000001be       0x64 USB10.o
                0x000001be                __vector_25
 .text.RemoveWhiteSpace
                0x00000222       0x1a USB10.o
                0x00000222                RemoveWhiteSpace
 .text.GetHexNumber
                0x0000023c       0x72 USB10.o
                0x0000023c                GetHexNumber
 .text.ParseNumber
                0x000002ae       0x6a USB10.o
                0x000002ae                ParseNumber
 .text.__vector_23
                0x00000318       0x56 USB10.o
                0x00000318                __vector_23
 .text.Command_Task
                0x0000036e      0x2e8 USB10.o
                0x0000036e                Command_Task
 .text.Event_USB_Disconnect
                0x00000656       0x10 USB10.o
                0x00000656                Event_USB_Disconnect
 .text.Event_USB_Connect
                0x00000666        0x8 USB10.o
                0x00000666                Event_USB_Connect
 .text.CDC_Task
                0x0000066e      0x1d0 USB10.o
                0x0000066e                CDC_Task
 .text.Event_USB_UnhandledControlPacket
                0x0000083e       0x80 USB10.o
                0x0000083e                Event_USB_UnhandledControlPacket
 .text.Event_USB_ConfigurationChanged
                0x000008be       0x2c USB10.o
                0x000008be                Event_USB_ConfigurationChanged
 .text.main     0x000008ea       0x72 USB10.o
                0x000008ea                main
 .text.USB_GetDescriptor
                0x0000095c       0x74 Descriptors.o
                0x0000095c                USB_GetDescriptor
 .text.Buffer_Initialize
                0x000009d0       0x28 RingBuff.o
                0x000009d0                Buffer_Initialize
 .text.Buffer_StoreElementOnTop
                0x000009f8       0x6e RingBuff.o
                0x000009f8                Buffer_StoreElementOnTop
 .text.Buffer_GetElementFromTop
                0x00000a66       0x5a RingBuff.o
                0x00000a66                Buffer_GetElementFromTop
 .text.Buffer_GetElementFromBottom
                0x00000ac0       0x60 RingBuff.o
                0x00000ac0                Buffer_GetElementFromBottom
 .text.Buffer_StoreElementOnBottom
                0x00000b20       0x52 RingBuff.o
                0x00000b20                Buffer_StoreElementOnBottom
 .text.I2C_Init
                0x00000b72        0xc I2C_bitbanged.o
                0x00000b72                I2C_Init
 .text.I2C_Get_ACK
                0x00000b7e       0x58 I2C_bitbanged.o
                0x00000b7e                I2C_Get_ACK
 .text.I2C_Start
                0x00000bd6       0x46 I2C_bitbanged.o
                0x00000bd6                I2C_Start
 .text.I2C_Stop
                0x00000c1c       0x64 I2C_bitbanged.o
                0x00000c1c                I2C_Stop
 .text.I2C_Pulse_SCL_After_ACK
                0x00000c80       0x4c I2C_bitbanged.o
                0x00000c80                I2C_Pulse_SCL_After_ACK
 .text.I2C_Pulse_SCL
                0x00000ccc       0x46 I2C_bitbanged.o
                0x00000ccc                I2C_Pulse_SCL
 .text.I2C_Send_NACK
                0x00000d12        0x4 I2C_bitbanged.o
                0x00000d12                I2C_Send_NACK
 .text.I2C_Send_ACK
                0x00000d16        0x8 I2C_bitbanged.o
                0x00000d16                I2C_Send_ACK
 .text.I2C_Send_Byte
                0x00000d1e       0x40 I2C_bitbanged.o
                0x00000d1e                I2C_Send_Byte
 .text.I2C_Write
                0x00000d5e       0x6c I2C_bitbanged.o
                0x00000d5e                I2C_Write
 .text.I2C_Receive_Byte
                0x00000dca       0x78 I2C_bitbanged.o
                0x00000dca                I2C_Receive_Byte
 .text.I2C_Read
                0x00000e42       0x70 I2C_bitbanged.o
                0x00000e42                I2C_Read
 .text.StepDirLineCoding_Init
                0x00000eb2        0xe StepDirLineCoding.o
                0x00000eb2                StepDirLineCoding_Init
 .text.StartCodition
                0x00000ec0       0x92 StepDirLineCoding.o
                0x00000ec0                StartCodition
 .text.SendByte
                0x00000f52      0x11c StepDirLineCoding.o
                0x00000f52                SendByte
 .text.Scheduler_SetTaskMode
                0x0000106e       0x32 ../../MyUSB/Scheduler/Scheduler.o
                0x0000106e                Scheduler_SetTaskMode
 .text.USB_SetupInterface
                0x000010a0       0xa6 ../../MyUSB/Drivers/USB/LowLevel/LowLevel.o
                0x000010a0                USB_SetupInterface
 .text.USB_ShutDown
                0x00001146       0x28 ../../MyUSB/Drivers/USB/LowLevel/LowLevel.o
                0x00001146                USB_ShutDown
 .text.USB_Init
                0x0000116e       0x16 ../../MyUSB/Drivers/USB/LowLevel/LowLevel.o
                0x0000116e                USB_Init
 .text.Endpoint_ConfigureEndpoint_P
                0x00001184       0x4e ../../MyUSB/Drivers/USB/LowLevel/Endpoint.o
                0x00001184                Endpoint_ConfigureEndpoint_P
 .text.Endpoint_Write_Control_Stream_LE
                0x000011d2       0x88 ../../MyUSB/Drivers/USB/LowLevel/Endpoint.o
                0x000011d2                Endpoint_Write_Control_Stream_LE
 .text.Endpoint_Read_Control_Stream_LE
                0x0000125a       0x3e ../../MyUSB/Drivers/USB/LowLevel/Endpoint.o
                0x0000125a                Endpoint_Read_Control_Stream_LE
 .text.USB_Device_ProcessControlPacket
                0x00001298      0x3a8 ../../MyUSB/Drivers/USB/LowLevel/DevChapter9.o
                0x00001298                USB_Device_ProcessControlPacket
 .text.USB_USBTask
                0x00001640       0x26 ../../MyUSB/Drivers/USB/HighLevel/USBTask.o
                0x00001640                USB_USBTask
 .text.USB_INT_DisableAllInterrupts
                0x00001666        0x6 ../../MyUSB/Drivers/USB/HighLevel/USBInterrupt.o
                0x00001666                USB_INT_DisableAllInterrupts
 .text.USB_INT_ClearAllInterrupts
                0x0000166c        0x6 ../../MyUSB/Drivers/USB/HighLevel/USBInterrupt.o
                0x0000166c                USB_INT_ClearAllInterrupts
 .text.__vector_11
                0x00001672      0x128 ../../MyUSB/Drivers/USB/HighLevel/USBInterrupt.o
                0x00001672                __vector_11
 .text.__stub   0x0000179a        0x2 ../../MyUSB/Drivers/USB/HighLevel/Events.o
                0x0000179a                Event_USB_DeviceError
                0x0000179a                Event_USB_Suspend
                0x0000179a                Event_USB_Reset
                0x0000179a                Event_USB_DeviceEnumerationComplete
                0x0000179a                Event_USB_WakeUp
 .text.libgcc   0x0000179c       0x24 c:/winavr-20080610/bin/../lib/gcc/avr/4.3.0/avr35\libgcc.a(_mulhi3.o)
                0x0000179c                __mulhi3
 .text.libgcc   0x000017c0       0x28 c:/winavr-20080610/bin/../lib/gcc/avr/4.3.0/avr35\libgcc.a(_udivmodhi4.o)
                0x000017c0                __udivmodhi4
 .text.libgcc   0x000017e8       0x44 c:/winavr-20080610/bin/../lib/gcc/avr/4.3.0/avr35\libgcc.a(_udivmodsi4.o)
                0x000017e8                __udivmodsi4
                0x0000182c                . = ALIGN (0x2)
 *(.fini9)
 .fini9         0x0000182c        0x0 c:/winavr-20080610/bin/../lib/gcc/avr/4.3.0/avr35\libgcc.a(_exit.o)
                0x0000182c                exit
                0x0000182c                _exit
 *(.fini9)
 *(.fini8)
 *(.fini8)
 *(.fini7)
 *(.fini7)
 *(.fini6)
 *(.fini6)
 *(.fini5)
 *(.fini5)
 *(.fini4)
 *(.fini4)
 *(.fini3)
 *(.fini3)
 *(.fini2)
 *(.fini2)
 *(.fini1)
 *(.fini1)
 *(.fini0)
 .fini0         0x0000182c        0x4 c:/winavr-20080610/bin/../lib/gcc/avr/4.3.0/avr35\libgcc.a(_exit.o)
 *(.fini0)
                0x00001830                _etext = .

.data           0x00800100       0x26 load address 0x00001830
                0x00800100                PROVIDE (__data_start, .)
 *(.data)
 .data          0x00800100       0x25 USB10.o
                0x00800113                bootloader
                0x0080010c                LineCoding
                0x00800100                Scheduler_TaskList
 .data          0x00800125        0x1 ../../MyUSB/Drivers/USB/LowLevel/Endpoint.o
                0x00800125                USB_ControlEndpointSize
 *(.data*)
 *(.rodata)
 *(.rodata*)
 *(.gnu.linkonce.d*)
                0x00800126                . = ALIGN (0x2)
                0x00800126                _edata = .
                0x00800126                PROVIDE (__data_end, .)

.bss            0x00800126      0x141 load address 0x00001856
                0x00800126                PROVIDE (__bss_start, .)
 *(.bss)
 .bss           0x00800126        0x7 USB10.o
                0x0080012b                outputBufferTail
                0x00800128                inputBufferHead
                0x00800127                escapeCharReceived
                0x00800129                inputBufferTail
                0x0080012c                mode
                0x0080012a                outputBufferHead
                0x00800126                Transmitting
 *(.bss*)
 *(COMMON)
 COMMON         0x0080012d      0x132 USB10.o
                0x0080012d                outputBuffer
                0x00800141                inputBuffer
                0x00800155                Tx_Buffer
                0x008001da                Rx_Buffer
 COMMON         0x0080025f        0x3 ../../MyUSB/Scheduler/Scheduler.o
                0x0080025f                Scheduler_TotalTasks
                0x00800260                Scheduler_TickCounter
 COMMON         0x00800262        0x3 ../../MyUSB/Drivers/USB/LowLevel/DevChapter9.o
                0x00800262                USB_CurrentlySelfPowered
                0x00800263                USB_RemoteWakeupEnabled
                0x00800264                USB_ConfigurationNumber
 COMMON         0x00800265        0x2 ../../MyUSB/Drivers/USB/HighLevel/USBTask.o
                0x00800265                USB_IsInitialized
                0x00800266                USB_IsConnected
                0x00800267                PROVIDE (__bss_end, .)
                0x00001830                __data_load_start = LOADADDR (.data)
                0x00001856                __data_load_end = (__data_load_start + SIZEOF (.data))

.noinit         0x00800267        0x0
                0x00800267                PROVIDE (__noinit_start, .)
 *(.noinit*)
                0x00800267                PROVIDE (__noinit_end, .)
                0x00800267                _end = .
                0x00800267                PROVIDE (__heap_start, .)

.eeprom         0x00810000        0x0
 *(.eeprom*)
                0x00810000                __eeprom_end = .

.fuse
 *(.fuse)
 *(.lfuse)
 *(.hfuse)
 *(.efuse)

.lock
 *(.lock*)

.signature
 *(.signature*)

.stab
 *(.stab)

.stabstr
 *(.stabstr)

.stab.excl
 *(.stab.excl)

.stab.exclstr
 *(.stab.exclstr)

.stab.index
 *(.stab.index)

.stab.indexstr
 *(.stab.indexstr)

.comment
 *(.comment)

.debug
 *(.debug)

.line
 *(.line)

.debug_srcinfo
 *(.debug_srcinfo)

.debug_sfnames
 *(.debug_sfnames)

.debug_aranges  0x00000000      0x368
 *(.debug_aranges)
 .debug_aranges
                0x00000000       0x98 USB10.o
 .debug_aranges
                0x00000098       0x20 Descriptors.o
 .debug_aranges
                0x000000b8       0x40 RingBuff.o
 .debug_aranges
                0x000000f8       0x88 I2C_bitbanged.o
 .debug_aranges
                0x00000180       0x30 StepDirLineCoding.o
 .debug_aranges
                0x000001b0       0x30 ../../MyUSB/Scheduler/Scheduler.o
 .debug_aranges
                0x000001e0       0x30 ../../MyUSB/Drivers/AT90USBXXX/Serial.o
 .debug_aranges
                0x00000210       0x30 ../../MyUSB/Drivers/USB/LowLevel/LowLevel.o
 .debug_aranges
                0x00000240       0x78 ../../MyUSB/Drivers/USB/LowLevel/Endpoint.o
 .debug_aranges
                0x000002b8       0x20 ../../MyUSB/Drivers/USB/LowLevel/DevChapter9.o
 .debug_aranges
                0x000002d8       0x20 ../../MyUSB/Drivers/USB/HighLevel/USBTask.o
 .debug_aranges
                0x000002f8       0x30 ../../MyUSB/Drivers/USB/HighLevel/USBInterrupt.o
 .debug_aranges
                0x00000328       0x20 ../../MyUSB/Drivers/USB/HighLevel/Events.o
 .debug_aranges
                0x00000348       0x20 ../../MyUSB/Drivers/USB/HighLevel/StdDescriptors.o

.debug_pubnames
                0x00000000      0x94b
 *(.debug_pubnames)
 .debug_pubnames
                0x00000000      0x294 USB10.o
 .debug_pubnames
                0x00000294       0x95 Descriptors.o
 .debug_pubnames
                0x00000329       0xa2 RingBuff.o
 .debug_pubnames
                0x000003cb       0xfd I2C_bitbanged.o
 .debug_pubnames
                0x000004c8       0x4c StepDirLineCoding.o
 .debug_pubnames
                0x00000514       0x9c ../../MyUSB/Scheduler/Scheduler.o
 .debug_pubnames
                0x000005b0       0x4c ../../MyUSB/Drivers/AT90USBXXX/Serial.o
 .debug_pubnames
                0x000005fc       0x47 ../../MyUSB/Drivers/USB/LowLevel/LowLevel.o
 .debug_pubnames
                0x00000643      0x1a7 ../../MyUSB/Drivers/USB/LowLevel/Endpoint.o
 .debug_pubnames
                0x000007ea       0x8b ../../MyUSB/Drivers/USB/LowLevel/DevChapter9.o
 .debug_pubnames
                0x00000875       0x4c ../../MyUSB/Drivers/USB/HighLevel/USBTask.o
 .debug_pubnames
                0x000008c1       0x62 ../../MyUSB/Drivers/USB/HighLevel/USBInterrupt.o
 .debug_pubnames
                0x00000923       0x28 ../../MyUSB/Drivers/USB/HighLevel/StdDescriptors.o

.debug_info     0x00000000     0x36ca
 *(.debug_info)
 .debug_info    0x00000000      0x8a7 USB10.o
 .debug_info    0x000008a7      0x718 Descriptors.o
 .debug_info    0x00000fbf      0x3ac RingBuff.o
 .debug_info    0x0000136b      0x552 I2C_bitbanged.o
 .debug_info    0x000018bd      0x114 StepDirLineCoding.o
 .debug_info    0x000019d1      0x2ab ../../MyUSB/Scheduler/Scheduler.o
 .debug_info    0x00001c7c      0x187 ../../MyUSB/Drivers/AT90USBXXX/Serial.o
 .debug_info    0x00001e03      0x35b ../../MyUSB/Drivers/USB/LowLevel/LowLevel.o
 .debug_info    0x0000215e      0x6a9 ../../MyUSB/Drivers/USB/LowLevel/Endpoint.o
 .debug_info    0x00002807      0x968 ../../MyUSB/Drivers/USB/LowLevel/DevChapter9.o
 .debug_info    0x0000316f      0x1a0 ../../MyUSB/Drivers/USB/HighLevel/USBTask.o
 .debug_info    0x0000330f      0x18d ../../MyUSB/Drivers/USB/HighLevel/USBInterrupt.o
 .debug_info    0x0000349c       0x7c ../../MyUSB/Drivers/USB/HighLevel/Events.o
 .debug_info    0x00003518      0x1b2 ../../MyUSB/Drivers/USB/HighLevel/StdDescriptors.o
 *(.gnu.linkonce.wi.*)

.debug_abbrev   0x00000000     0x1349
 *(.debug_abbrev)
 .debug_abbrev  0x00000000      0x2f4 USB10.o
 .debug_abbrev  0x000002f4      0x16b Descriptors.o
 .debug_abbrev  0x0000045f      0x183 RingBuff.o
 .debug_abbrev  0x000005e2      0x18e I2C_bitbanged.o
 .debug_abbrev  0x00000770       0xb6 StepDirLineCoding.o
 .debug_abbrev  0x00000826      0x179 ../../MyUSB/Scheduler/Scheduler.o
 .debug_abbrev  0x0000099f       0xf7 ../../MyUSB/Drivers/AT90USBXXX/Serial.o
 .debug_abbrev  0x00000a96      0x144 ../../MyUSB/Drivers/USB/LowLevel/LowLevel.o
 .debug_abbrev  0x00000bda      0x23e ../../MyUSB/Drivers/USB/LowLevel/Endpoint.o
 .debug_abbrev  0x00000e18      0x258 ../../MyUSB/Drivers/USB/LowLevel/DevChapter9.o
 .debug_abbrev  0x00001070       0xfe ../../MyUSB/Drivers/USB/HighLevel/USBTask.o
 .debug_abbrev  0x0000116e       0xba ../../MyUSB/Drivers/USB/HighLevel/USBInterrupt.o
 .debug_abbrev  0x00001228       0x3f ../../MyUSB/Drivers/USB/HighLevel/Events.o
 .debug_abbrev  0x00001267       0xe2 ../../MyUSB/Drivers/USB/HighLevel/StdDescriptors.o

.debug_line     0x00000000     0x3203
 *(.debug_line)
 .debug_line    0x00000000      0xba6 USB10.o
 .debug_line    0x00000ba6      0x19d Descriptors.o
 .debug_line    0x00000d43      0x345 RingBuff.o
 .debug_line    0x00001088      0x5c9 I2C_bitbanged.o
 .debug_line    0x00001651      0x1f3 StepDirLineCoding.o
 .debug_line    0x00001844      0x1e9 ../../MyUSB/Scheduler/Scheduler.o
 .debug_line    0x00001a2d      0x16b ../../MyUSB/Drivers/AT90USBXXX/Serial.o
 .debug_line    0x00001b98      0x2fe ../../MyUSB/Drivers/USB/LowLevel/LowLevel.o
 .debug_line    0x00001e96      0x6b6 ../../MyUSB/Drivers/USB/LowLevel/Endpoint.o
 .debug_line    0x0000254c      0x5d6 ../../MyUSB/Drivers/USB/LowLevel/DevChapter9.o
 .debug_line    0x00002b22      0x154 ../../MyUSB/Drivers/USB/HighLevel/USBTask.o
 .debug_line    0x00002c76      0x363 ../../MyUSB/Drivers/USB/HighLevel/USBInterrupt.o
 .debug_line    0x00002fd9       0x89 ../../MyUSB/Drivers/USB/HighLevel/Events.o
 .debug_line    0x00003062      0x1a1 ../../MyUSB/Drivers/USB/HighLevel/StdDescriptors.o

.debug_frame    0x00000000      0x510
 *(.debug_frame)
 .debug_frame   0x00000000      0x110 USB10.o
 .debug_frame   0x00000110       0x20 Descriptors.o
 .debug_frame   0x00000130       0x60 RingBuff.o
 .debug_frame   0x00000190       0xf0 I2C_bitbanged.o
 .debug_frame   0x00000280       0x40 StepDirLineCoding.o
 .debug_frame   0x000002c0       0x40 ../../MyUSB/Scheduler/Scheduler.o
 .debug_frame   0x00000300       0x40 ../../MyUSB/Drivers/AT90USBXXX/Serial.o
 .debug_frame   0x00000340       0x40 ../../MyUSB/Drivers/USB/LowLevel/LowLevel.o
 .debug_frame   0x00000380       0xd0 ../../MyUSB/Drivers/USB/LowLevel/Endpoint.o
 .debug_frame   0x00000450       0x20 ../../MyUSB/Drivers/USB/LowLevel/DevChapter9.o
 .debug_frame   0x00000470       0x20 ../../MyUSB/Drivers/USB/HighLevel/USBTask.o
 .debug_frame   0x00000490       0x40 ../../MyUSB/Drivers/USB/HighLevel/USBInterrupt.o
 .debug_frame   0x000004d0       0x20 ../../MyUSB/Drivers/USB/HighLevel/Events.o
 .debug_frame   0x000004f0       0x20 ../../MyUSB/Drivers/USB/HighLevel/StdDescriptors.o

.debug_str      0x00000000     0x15d5
 *(.debug_str)
 .debug_str     0x00000000      0x545 USB10.o
                                0x5a2 (size before relaxing)
 .debug_str     0x00000545      0x48b Descriptors.o
                                0x647 (size before relaxing)
 .debug_str     0x000009d0       0xb9 RingBuff.o
                                0x1a3 (size before relaxing)
 .debug_str     0x00000a89       0xd2 I2C_bitbanged.o
                                0x1a4 (size before relaxing)
 .debug_str     0x00000b5b       0x65 StepDirLineCoding.o
                                0x119 (size before relaxing)
 .debug_str     0x00000bc0       0xa0 ../../MyUSB/Scheduler/Scheduler.o
                                0x21f (size before relaxing)
 .debug_str     0x00000c60       0x77 ../../MyUSB/Drivers/AT90USBXXX/Serial.o
                                0x167 (size before relaxing)
 .debug_str     0x00000cd7       0xf6 ../../MyUSB/Drivers/USB/LowLevel/LowLevel.o
                                0x3fb (size before relaxing)
 .debug_str     0x00000dcd      0x3f2 ../../MyUSB/Drivers/USB/LowLevel/Endpoint.o
                                0x5a8 (size before relaxing)
 .debug_str     0x000011bf      0x2ac ../../MyUSB/Drivers/USB/LowLevel/DevChapter9.o
                                0x716 (size before relaxing)
 .debug_str     0x0000146b       0x54 ../../MyUSB/Drivers/USB/HighLevel/USBTask.o
                                0x1bd (size before relaxing)
 .debug_str     0x000014bf       0x75 ../../MyUSB/Drivers/USB/HighLevel/USBInterrupt.o
                                0x1fc (size before relaxing)
 .debug_str     0x00001534       0x32 ../../MyUSB/Drivers/USB/HighLevel/Events.o
                                 0xde (size before relaxing)
 .debug_str     0x00001566       0x6f ../../MyUSB/Drivers/USB/HighLevel/StdDescriptors.o
                                0x1f7 (size before relaxing)

.debug_loc      0x00000000     0x13a0
 *(.debug_loc)
 .debug_loc     0x00000000      0x4c6 USB10.o
 .debug_loc     0x000004c6      0x178 Descriptors.o
 .debug_loc     0x0000063e       0xf9 RingBuff.o
 .debug_loc     0x00000737      0x25a I2C_bitbanged.o
 .debug_loc     0x00000991       0xa9 StepDirLineCoding.o
 .debug_loc     0x00000a3a       0xe1 ../../MyUSB/Scheduler/Scheduler.o
 .debug_loc     0x00000b1b       0x7e ../../MyUSB/Drivers/AT90USBXXX/Serial.o
 .debug_loc     0x00000b99       0x37 ../../MyUSB/Drivers/USB/LowLevel/LowLevel.o
 .debug_loc     0x00000bd0      0x463 ../../MyUSB/Drivers/USB/LowLevel/Endpoint.o
 .debug_loc     0x00001033      0x312 ../../MyUSB/Drivers/USB/LowLevel/DevChapter9.o
 .debug_loc     0x00001345       0x5b ../../MyUSB/Drivers/USB/HighLevel/StdDescriptors.o

.debug_macinfo
 *(.debug_macinfo)
OUTPUT(USB10.elf elf32-avr)
LOAD linker stubs

.debug_ranges   0x00000000      0x3d0
 .debug_ranges  0x00000000       0x90 USB10.o
 .debug_ranges  0x00000090       0x18 Descriptors.o
 .debug_ranges  0x000000a8       0x38 RingBuff.o
 .debug_ranges  0x000000e0       0x80 I2C_bitbanged.o
 .debug_ranges  0x00000160       0x28 StepDirLineCoding.o
 .debug_ranges  0x00000188       0x28 ../../MyUSB/Scheduler/Scheduler.o
 .debug_ranges  0x000001b0       0x28 ../../MyUSB/Drivers/AT90USBXXX/Serial.o
 .debug_ranges  0x000001d8       0x28 ../../MyUSB/Drivers/USB/LowLevel/LowLevel.o
 .debug_ranges  0x00000200       0x70 ../../MyUSB/Drivers/USB/LowLevel/Endpoint.o
 .debug_ranges  0x00000270       0xf0 ../../MyUSB/Drivers/USB/LowLevel/DevChapter9.o
 .debug_ranges  0x00000360       0x18 ../../MyUSB/Drivers/USB/HighLevel/USBTask.o
 .debug_ranges  0x00000378       0x28 ../../MyUSB/Drivers/USB/HighLevel/USBInterrupt.o
 .debug_ranges  0x000003a0       0x18 ../../MyUSB/Drivers/USB/HighLevel/Events.o
 .debug_ranges  0x000003b8       0x18 ../../MyUSB/Drivers/USB/HighLevel/StdDescriptors.o

Cross Reference Table

Symbol                                            File
BUTTTAG_BuildDate                                 USB10.o
BUTTTAG_BuildTime                                 USB10.o
BUTTTAG_MyUSBVersion                              USB10.o
BUTTTAG_ProjName                                  USB10.o
Buffer_GetElementFromBottom                       RingBuff.o
                                                  USB10.o
Buffer_GetElementFromTop                          RingBuff.o
                                                  USB10.o
Buffer_Initialize                                 RingBuff.o
                                                  USB10.o
Buffer_StoreElementOnBottom                       RingBuff.o
                                                  USB10.o
Buffer_StoreElementOnTop                          RingBuff.o
                                                  USB10.o
CDC_Task                                          USB10.o
Command_Task                                      USB10.o
ConfigurationDescriptor                           Descriptors.o
Delay                                             I2C_bitbanged.o
DeviceDescriptor                                  Descriptors.o
Endpoint_ClearEndpoints                           ../../MyUSB/Drivers/USB/LowLevel/Endpoint.o
Endpoint_ConfigureEndpoint_P                      ../../MyUSB/Drivers/USB/LowLevel/Endpoint.o
                                                  ../../MyUSB/Drivers/USB/HighLevel/USBInterrupt.o
                                                  USB10.o
Endpoint_Discard_Stream                           ../../MyUSB/Drivers/USB/LowLevel/Endpoint.o
Endpoint_Read_Control_Stream_BE                   ../../MyUSB/Drivers/USB/LowLevel/Endpoint.o
Endpoint_Read_Control_Stream_LE                   ../../MyUSB/Drivers/USB/LowLevel/Endpoint.o
                                                  USB10.o
Endpoint_Read_Stream_BE                           ../../MyUSB/Drivers/USB/LowLevel/Endpoint.o
Endpoint_Read_Stream_LE                           ../../MyUSB/Drivers/USB/LowLevel/Endpoint.o
Endpoint_WaitUntilReady                           ../../MyUSB/Drivers/USB/LowLevel/Endpoint.o
Endpoint_Write_Control_Stream_BE                  ../../MyUSB/Drivers/USB/LowLevel/Endpoint.o
Endpoint_Write_Control_Stream_LE                  ../../MyUSB/Drivers/USB/LowLevel/Endpoint.o
                                                  USB10.o
Endpoint_Write_Stream_BE                          ../../MyUSB/Drivers/USB/LowLevel/Endpoint.o
Endpoint_Write_Stream_LE                          ../../MyUSB/Drivers/USB/LowLevel/Endpoint.o
Event_USB_ConfigurationChanged                    USB10.o
                                                  ../../MyUSB/Drivers/USB/LowLevel/DevChapter9.o
Event_USB_Connect                                 USB10.o
                                                  ../../MyUSB/Drivers/USB/HighLevel/USBInterrupt.o
Event_USB_DeviceEnumerationComplete               ../../MyUSB/Drivers/USB/HighLevel/Events.o
                                                  ../../MyUSB/Drivers/USB/LowLevel/DevChapter9.o
Event_USB_DeviceError                             ../../MyUSB/Drivers/USB/HighLevel/Events.o
                                                  ../../MyUSB/Drivers/USB/HighLevel/StdDescriptors.o
Event_USB_Disconnect                              USB10.o
                                                  ../../MyUSB/Drivers/USB/HighLevel/USBInterrupt.o
                                                  ../../MyUSB/Drivers/USB/LowLevel/LowLevel.o
Event_USB_Reset                                   ../../MyUSB/Drivers/USB/HighLevel/Events.o
                                                  ../../MyUSB/Drivers/USB/HighLevel/USBInterrupt.o
Event_USB_Suspend                                 ../../MyUSB/Drivers/USB/HighLevel/Events.o
                                                  ../../MyUSB/Drivers/USB/HighLevel/USBInterrupt.o
Event_USB_UnhandledControlPacket                  USB10.o
                                                  ../../MyUSB/Drivers/USB/LowLevel/DevChapter9.o
Event_USB_WakeUp                                  ../../MyUSB/Drivers/USB/HighLevel/Events.o
                                                  ../../MyUSB/Drivers/USB/HighLevel/USBInterrupt.o
GetHexNumber                                      USB10.o
I2C_Get_ACK                                       I2C_bitbanged.o
I2C_Init                                          I2C_bitbanged.o
                                                  USB10.o
I2C_Pulse_SCL                                     I2C_bitbanged.o
I2C_Pulse_SCL_After_ACK                           I2C_bitbanged.o
I2C_Read                                          I2C_bitbanged.o
                                                  USB10.o
I2C_Receive_Byte                                  I2C_bitbanged.o
I2C_RepeatedStart                                 I2C_bitbanged.o
I2C_Send_ACK                                      I2C_bitbanged.o
I2C_Send_Byte                                     I2C_bitbanged.o
I2C_Send_NACK                                     I2C_bitbanged.o
I2C_Start                                         I2C_bitbanged.o
I2C_Stop                                          I2C_bitbanged.o
I2C_Write                                         I2C_bitbanged.o
                                                  USB10.o
LanguageString                                    Descriptors.o
LineCoding                                        USB10.o
ManufacturerString                                Descriptors.o
ParseNumber                                       USB10.o
Print_Int                                         USB10.o
ProductString                                     Descriptors.o
ReconfigureUSART                                  USB10.o
RemoveWhiteSpace                                  USB10.o
Rx_Buffer                                         USB10.o
Scheduler_HasDelayElapsed                         ../../MyUSB/Scheduler/Scheduler.o
Scheduler_SetGroupTaskMode                        ../../MyUSB/Scheduler/Scheduler.o
Scheduler_SetTaskMode                             ../../MyUSB/Scheduler/Scheduler.o
                                                  USB10.o
Scheduler_TaskList                                USB10.o
                                                  ../../MyUSB/Scheduler/Scheduler.o
Scheduler_TickCounter                             ../../MyUSB/Scheduler/Scheduler.o
Scheduler_TotalTasks                              ../../MyUSB/Scheduler/Scheduler.o
                                                  USB10.o
SendByte                                          StepDirLineCoding.o
                                                  USB10.o
Serial_Init                                       ../../MyUSB/Drivers/AT90USBXXX/Serial.o
Serial_TxString                                   ../../MyUSB/Drivers/AT90USBXXX/Serial.o
Serial_TxString_P                                 ../../MyUSB/Drivers/AT90USBXXX/Serial.o
StartCodition                                     StepDirLineCoding.o
StepDirLineCoding_Init                            StepDirLineCoding.o
                                                  USB10.o
Transmitting                                      USB10.o
Tx_Buffer                                         USB10.o
USB_ConfigurationNumber                           ../../MyUSB/Drivers/USB/HighLevel/USBInterrupt.o
                                                  ../../MyUSB/Drivers/USB/LowLevel/DevChapter9.o
                                                  ../../MyUSB/Drivers/USB/LowLevel/LowLevel.o
USB_ControlEndpointSize                           ../../MyUSB/Drivers/USB/LowLevel/Endpoint.o
                                                  ../../MyUSB/Drivers/USB/HighLevel/USBInterrupt.o
                                                  ../../MyUSB/Drivers/USB/LowLevel/DevChapter9.o
                                                  ../../MyUSB/Drivers/USB/LowLevel/LowLevel.o
USB_CurrentlySelfPowered                          ../../MyUSB/Drivers/USB/LowLevel/DevChapter9.o
                                                  ../../MyUSB/Drivers/USB/LowLevel/LowLevel.o
USB_Device_ProcessControlPacket                   ../../MyUSB/Drivers/USB/LowLevel/DevChapter9.o
                                                  ../../MyUSB/Drivers/USB/HighLevel/USBTask.o
USB_GetDescriptor                                 Descriptors.o
                                                  ../../MyUSB/Drivers/USB/LowLevel/DevChapter9.o
                                                  ../../MyUSB/Drivers/USB/LowLevel/LowLevel.o
USB_INT_ClearAllInterrupts                        ../../MyUSB/Drivers/USB/HighLevel/USBInterrupt.o
                                                  ../../MyUSB/Drivers/USB/LowLevel/LowLevel.o
USB_INT_DisableAllInterrupts                      ../../MyUSB/Drivers/USB/HighLevel/USBInterrupt.o
                                                  ../../MyUSB/Drivers/USB/LowLevel/LowLevel.o
USB_Init                                          ../../MyUSB/Drivers/USB/LowLevel/LowLevel.o
                                                  USB10.o
USB_IsConnected                                   ../../MyUSB/Drivers/USB/HighLevel/USBInterrupt.o
                                                  ../../MyUSB/Drivers/USB/HighLevel/USBTask.o
                                                  ../../MyUSB/Drivers/USB/LowLevel/Endpoint.o
                                                  ../../MyUSB/Drivers/USB/LowLevel/LowLevel.o
                                                  USB10.o
USB_IsInitialized                                 ../../MyUSB/Drivers/USB/HighLevel/USBTask.o
                                                  ../../MyUSB/Drivers/USB/LowLevel/LowLevel.o
USB_RemoteWakeupEnabled                           ../../MyUSB/Drivers/USB/LowLevel/DevChapter9.o
                                                  ../../MyUSB/Drivers/USB/LowLevel/LowLevel.o
USB_SetupInterface                                ../../MyUSB/Drivers/USB/LowLevel/LowLevel.o
USB_ShutDown                                      ../../MyUSB/Drivers/USB/LowLevel/LowLevel.o
USB_USBTask                                       ../../MyUSB/Drivers/USB/HighLevel/USBTask.o
                                                  USB10.o
__bad_interrupt                                   c:/winavr-20080610/bin/../lib/gcc/avr/4.3.0/../../../../avr/lib/avr35/crtusb162.o
__bss_end                                         c:/winavr-20080610/bin/../lib/gcc/avr/4.3.0/avr35\libgcc.a(_clear_bss.o)
__bss_start                                       c:/winavr-20080610/bin/../lib/gcc/avr/4.3.0/avr35\libgcc.a(_clear_bss.o)
__data_end                                        c:/winavr-20080610/bin/../lib/gcc/avr/4.3.0/avr35\libgcc.a(_copy_data.o)
__data_load_start                                 c:/winavr-20080610/bin/../lib/gcc/avr/4.3.0/avr35\libgcc.a(_copy_data.o)
__data_start                                      c:/winavr-20080610/bin/../lib/gcc/avr/4.3.0/avr35\libgcc.a(_copy_data.o)
__do_clear_bss                                    c:/winavr-20080610/bin/../lib/gcc/avr/4.3.0/avr35\libgcc.a(_clear_bss.o)
                                                  ../../MyUSB/Drivers/USB/HighLevel/StdDescriptors.o
                                                  ../../MyUSB/Drivers/USB/HighLevel/Events.o
                                                  ../../MyUSB/Drivers/USB/HighLevel/USBInterrupt.o
                                                  ../../MyUSB/Drivers/USB/HighLevel/USBTask.o
                                                  ../../MyUSB/Drivers/USB/LowLevel/DevChapter9.o
                                                  ../../MyUSB/Drivers/USB/LowLevel/Endpoint.o
                                                  ../../MyUSB/Drivers/USB/LowLevel/LowLevel.o
                                                  ../../MyUSB/Drivers/AT90USBXXX/Serial.o
                                                  ../../MyUSB/Scheduler/Scheduler.o
                                                  StepDirLineCoding.o
                                                  I2C_bitbanged.o
                                                  RingBuff.o
                                                  Descriptors.o
                                                  USB10.o
__do_copy_data                                    c:/winavr-20080610/bin/../lib/gcc/avr/4.3.0/avr35\libgcc.a(_copy_data.o)
                                                  ../../MyUSB/Drivers/USB/HighLevel/StdDescriptors.o
                                                  ../../MyUSB/Drivers/USB/HighLevel/Events.o
                                                  ../../MyUSB/Drivers/USB/HighLevel/USBInterrupt.o
                                                  ../../MyUSB/Drivers/USB/HighLevel/USBTask.o
                                                  ../../MyUSB/Drivers/USB/LowLevel/DevChapter9.o
                                                  ../../MyUSB/Drivers/USB/LowLevel/Endpoint.o
                                                  ../../MyUSB/Drivers/USB/LowLevel/LowLevel.o
                                                  ../../MyUSB/Drivers/AT90USBXXX/Serial.o
                                                  ../../MyUSB/Scheduler/Scheduler.o
                                                  StepDirLineCoding.o
                                                  I2C_bitbanged.o
                                                  RingBuff.o
                                                  Descriptors.o
                                                  USB10.o
__heap_end                                        c:/winavr-20080610/bin/../lib/gcc/avr/4.3.0/../../../../avr/lib/avr35/crtusb162.o
__init                                            c:/winavr-20080610/bin/../lib/gcc/avr/4.3.0/../../../../avr/lib/avr35/crtusb162.o
__mulhi3                                          c:/winavr-20080610/bin/../lib/gcc/avr/4.3.0/avr35\libgcc.a(_mulhi3.o)
                                                  USB10.o
__stack                                           c:/winavr-20080610/bin/../lib/gcc/avr/4.3.0/../../../../avr/lib/avr35/crtusb162.o
__udivmodhi4                                      c:/winavr-20080610/bin/../lib/gcc/avr/4.3.0/avr35\libgcc.a(_udivmodhi4.o)
                                                  ../../MyUSB/Drivers/USB/LowLevel/DevChapter9.o
                                                  ../../MyUSB/Drivers/USB/LowLevel/Endpoint.o
                                                  USB10.o
__udivmodsi4                                      c:/winavr-20080610/bin/../lib/gcc/avr/4.3.0/avr35\libgcc.a(_udivmodsi4.o)
                                                  ../../MyUSB/Drivers/AT90USBXXX/Serial.o
                                                  USB10.o
__vector_1                                        c:/winavr-20080610/bin/../lib/gcc/avr/4.3.0/../../../../avr/lib/avr35/crtusb162.o
__vector_10                                       c:/winavr-20080610/bin/../lib/gcc/avr/4.3.0/../../../../avr/lib/avr35/crtusb162.o
__vector_11                                       ../../MyUSB/Drivers/USB/HighLevel/USBInterrupt.o
                                                  c:/winavr-20080610/bin/../lib/gcc/avr/4.3.0/../../../../avr/lib/avr35/crtusb162.o
__vector_12                                       c:/winavr-20080610/bin/../lib/gcc/avr/4.3.0/../../../../avr/lib/avr35/crtusb162.o
__vector_13                                       c:/winavr-20080610/bin/../lib/gcc/avr/4.3.0/../../../../avr/lib/avr35/crtusb162.o
__vector_14                                       c:/winavr-20080610/bin/../lib/gcc/avr/4.3.0/../../../../avr/lib/avr35/crtusb162.o
__vector_15                                       c:/winavr-20080610/bin/../lib/gcc/avr/4.3.0/../../../../avr/lib/avr35/crtusb162.o
__vector_16                                       c:/winavr-20080610/bin/../lib/gcc/avr/4.3.0/../../../../avr/lib/avr35/crtusb162.o
__vector_17                                       c:/winavr-20080610/bin/../lib/gcc/avr/4.3.0/../../../../avr/lib/avr35/crtusb162.o
__vector_18                                       c:/winavr-20080610/bin/../lib/gcc/avr/4.3.0/../../../../avr/lib/avr35/crtusb162.o
__vector_19                                       c:/winavr-20080610/bin/../lib/gcc/avr/4.3.0/../../../../avr/lib/avr35/crtusb162.o
__vector_2                                        c:/winavr-20080610/bin/../lib/gcc/avr/4.3.0/../../../../avr/lib/avr35/crtusb162.o
__vector_20                                       c:/winavr-20080610/bin/../lib/gcc/avr/4.3.0/../../../../avr/lib/avr35/crtusb162.o
__vector_21                                       c:/winavr-20080610/bin/../lib/gcc/avr/4.3.0/../../../../avr/lib/avr35/crtusb162.o
__vector_22                                       c:/winavr-20080610/bin/../lib/gcc/avr/4.3.0/../../../../avr/lib/avr35/crtusb162.o
__vector_23                                       USB10.o
                                                  c:/winavr-20080610/bin/../lib/gcc/avr/4.3.0/../../../../avr/lib/avr35/crtusb162.o
__vector_24                                       c:/winavr-20080610/bin/../lib/gcc/avr/4.3.0/../../../../avr/lib/avr35/crtusb162.o
__vector_25                                       USB10.o
                                                  c:/winavr-20080610/bin/../lib/gcc/avr/4.3.0/../../../../avr/lib/avr35/crtusb162.o
__vector_26                                       c:/winavr-20080610/bin/../lib/gcc/avr/4.3.0/../../../../avr/lib/avr35/crtusb162.o
__vector_27                                       c:/winavr-20080610/bin/../lib/gcc/avr/4.3.0/../../../../avr/lib/avr35/crtusb162.o
__vector_28                                       c:/winavr-20080610/bin/../lib/gcc/avr/4.3.0/../../../../avr/lib/avr35/crtusb162.o
__vector_3                                        c:/winavr-20080610/bin/../lib/gcc/avr/4.3.0/../../../../avr/lib/avr35/crtusb162.o
__vector_4                                        c:/winavr-20080610/bin/../lib/gcc/avr/4.3.0/../../../../avr/lib/avr35/crtusb162.o
__vector_5                                        c:/winavr-20080610/bin/../lib/gcc/avr/4.3.0/../../../../avr/lib/avr35/crtusb162.o
__vector_6                                        c:/winavr-20080610/bin/../lib/gcc/avr/4.3.0/../../../../avr/lib/avr35/crtusb162.o
__vector_7                                        c:/winavr-20080610/bin/../lib/gcc/avr/4.3.0/../../../../avr/lib/avr35/crtusb162.o
__vector_8                                        c:/winavr-20080610/bin/../lib/gcc/avr/4.3.0/../../../../avr/lib/avr35/crtusb162.o
__vector_9                                        c:/winavr-20080610/bin/../lib/gcc/avr/4.3.0/../../../../avr/lib/avr35/crtusb162.o
__vector_default                                  c:/winavr-20080610/bin/../lib/gcc/avr/4.3.0/../../../../avr/lib/avr35/crtusb162.o
__vectors                                         c:/winavr-20080610/bin/../lib/gcc/avr/4.3.0/../../../../avr/lib/avr35/crtusb162.o
_exit                                             c:/winavr-20080610/bin/../lib/gcc/avr/4.3.0/avr35\libgcc.a(_exit.o)
bootloader                                        USB10.o
escapeCharReceived                                USB10.o
exit                                              c:/winavr-20080610/bin/../lib/gcc/avr/4.3.0/avr35\libgcc.a(_exit.o)
                                                  c:/winavr-20080610/bin/../lib/gcc/avr/4.3.0/../../../../avr/lib/avr35/crtusb162.o
inputBuffer                                       USB10.o
inputBufferHead                                   USB10.o
inputBufferTail                                   USB10.o
main                                              USB10.o
                                                  c:/winavr-20080610/bin/../lib/gcc/avr/4.3.0/../../../../avr/lib/avr35/crtusb162.o
mode                                              USB10.o
outputBuffer                                      USB10.o
outputBufferHead                                  USB10.o
outputBufferTail                                  USB10.o
testReset                                         USB10.o
uart_puts                                         USB10.o
